:020000040000FA
:10000000000000008A011908A0000730990085014E
:1000100083169F01C8308500831203012620200823
:100020001F39073A03191F288316FF23831226203E
:10003000851603303C20851203303C201828051615
:1000400003303C20051203303C201F280511A3007B
:1000500085100830A2000510A30D03180514000038
:10006000851400008510A20B2B2805150800A4009C
:100070004220A40B38280800A50064303720A50BC7
:100080003D280800C6300000FF3E031D4328000045
:1000900000000000080043346F3470347934723447
:1000A00069346734683474342034503465347434BB
:1000B00065342034473472346934663466346934C4
:1000C000743468347334203428344334293420346D
:1000D00032343034303438342034313432344634ED
:1000E0003634323439342F343634373435342034DE
:1000F0004F3453344334433441344C342034743417
:1001000065347334743420347534743469346C3425
:10011000693474347934203431342E34303430340A
:10012000203468347434743470343A342F342F34B7
:10013000703469346334703472346F346A346534C3
:100140006334743473342E346F34723467342E3421
:0601500075346B3420340D
:02400E00A43FCD
:00000001FF
